:020000040801F1
:1000000038410020A1010108931A01086318010872
:10001000911A01081D090108D11F01080000000004
:10002000000000000000000000000000971A010816
:100030001F09010800000000951A0108991A01081B
:10004000BB010108BB010108BB010108BB0101089C
:10005000BB010108BB010108BB010108BB0101088C
:10006000BB010108BB010108BB010108BB0101087C
:10007000BB010108BB010108BB010108BB0101086C
:10008000BB010108BB010108BB010108BB0101085C
:10009000BB010108BB010108BB010108BB0101084C
:1000A000BB010108BB010108BB010108BB0101083C
:1000B000BB010108BB010108BB010108BB0101082C
:1000C000BB010108BB010108BB010108BB0101081C
:1000D000BB010108B91F0108C51F0108BB010108C8
:1000E000BB010108BB010108BB010108BB010108FC
:1000F000BB010108BB010108BB010108BB010108EC
:10010000BB010108BB010108BB010108BB010108DB
:10011000751B0108BB010108BB010108BB010108F7
:10012000BB010108BB010108BB010108BB010108BB
:10013000BB010108BB010108BB010108BB010108AB
:10014000BB010108BB010108BB010108BB0101089B
:10015000BB010108BB010108BB010108BB0101088B
:10016000BB010108BB010108BB010108BB0101087B
:10017000BB010108BB010108BB0101080000000030
:10018000BB010108BB010108DFF810D000F020FB23
:1001900000480047D9280108AFF30080384100200B
:1001A0000648804706480047FEE7FEE7FEE7FEE711
:1001B000FEE7FEE7FEE7FEE7FEE7FEE71D1B0108A0
:1001C000890101082DE9F05F0546002092469B4613
:1001D00088460646814640241BE02846414647465D
:1001E000224600F00EFA53465A46C01A914110D3E7
:1001F00011461846224600F0F5F92D1A67EB010862
:100200004F4622460120002100F0ECF917EB0009CF
:100210004E41201EA4F10104DFDC484631462A4647
:100220004346BDE8F09FD2B201E000F8012B491E21
:10023000FBD270470022F6E710B513460A46044683
:100240001946FFF7F0FF204610BD2DE9FE4F80460E
:1002500081EA0300C00F0C46009021F0004123F01A
:100260000045B8EB0200A94105D240462146904620
:100270001C460B46024623F00040104347D0270D92
:10028000C7F30A00C3F30A510290401A01904028B4
:100290006BDAC3F3130040F4801B0098924620B140
:1002A0000023D2EB030A63EB0B0B01985946C0F114
:1002B0004002504600F096F906460D465046594613
:1002C000019A00F0AEF910EB08006141002487EAC2
:1002D000115284EAE7731A4340D0009A62B3019A3C
:1002E000012A4FEA075215DC001B61EB02014FF0B7
:1002F000004202EA0752CDE90042001C41F580119C
:1003000032462B4600F0E5F903B0BDE8F08F4046D9
:100310002146F9E7001B61EB0201001C41F5801347
:1003200000185B412018A2F5001747EB030140EAD3
:10033000D570B6196D4111E06D084FEA360645EAF1
:10034000C0754FEA0752001B61EB0201001C41F52A
:10035000801149084FEA30000019514132462B46BE
:1003600003B0BDE8F04F00F0A5B9009801224000AD
:100370000023D0EB020263EBE073009821464FEAC2
:10038000E074B8EB000061EB0401E9E783F000439F
:100390005BE781F0004158E72DE9FE4F81EA030455
:1003A00004F0004421F0004100944FF0000B23F0D2
:1003B000004350EA01045ED052EA03045BD0C3F369
:1003C0000A54C1F30A552C44A4F2F3340194A0FB5F
:1003D0000254C1F3130141F48011C3F3130343F436
:1003E000801301FB024400FB034E840A970A44EA8F
:1003F000815447EA8357A4FB076802958D0A05FBE1
:1004000007854FEA932C04FB0C542705029D4FEA05
:10041000065847EA1637B5EB08056EEB070C870E52
:10042000920E47EA811742EA8312A7FB0201B6EB5C
:100430000B0164EB00042B0D43EA0C335E1844EB14
:100440001C50DA465146E7FB0201C5F313044FEA9C
:100450000B3343EA14534FEA0432019C43EA060388
:10046000A4F10C040294009CCDE900B400F031F931
:1004700003B0BDE8F08F00200146F9E72DE9F04D0B
:1004800081EA030404F0004B21F0004514464FF0CC
:10049000000A23F0004150EA050220D054EA01028C
:1004A0001DD0C5F30A570246C5F31303C1F3130069
:1004B000C1F30A5640F4801543F48013A7EB0608F5
:1004C000101BD64608F2FD3873EB050002D308F185
:1004D000010801E092185B41B8F1000F03DA002037
:1004E0000146BDE8F08D00204FF480110646844699
:1004F0000EE0171B73EB050705D3121B63EB050317
:1005000006434CEA010C49084FEA300092185B415F
:1005100050EA0107EDD152EA030012D082EA04004A
:1005200083EA0501084305D0101BAB4106D2012226
:10053000002306E000224FF0004302E06FF00102CA
:1005400053101AEB06004CEB085110EB0A0041EB7C
:100550000B01BDE8F04D00F0ADB800F0004230F006
:1005600000400AD0C10D01F56071C0F3160042EAE7
:100570000151C208400711437047002001467047EF
:1005800001F0004330B421F0004150EA010206D0EE
:100590000A0DA2F56072C1F31301002A02DC30BC1F
:1005A00000207047440F44EAC104C100E01830BC89
:1005B00000EBC25000F047B830B50B4601460020B2
:1005C0002022012409E021FA02F59D4205D303FA15
:1005D00002F5491B04FA02F52844151EA2F1010296
:1005E000F1DC30BD202A04DB203A00FA02F10020C1
:1005F00070479140C2F1200320FA03F31943904061
:100600007047202A04DB203A21FA02F000217047CB
:1006100021FA02F3D040C2F120029140084319466A
:100620007047202A06DBCB17203A41FA02F043EA52
:10063000E07306E041FA02F3D040C2F1200291409B
:100640000843194670470029A8BF7047401C49005D
:1006500008BF20F00100704710B4B0FA80FC00FA27
:100660000CF050EA010404BF10BC704749B1CCF152
:10067000200421FA04F411FA0CF118BF01212143DE
:100680000843A3EB0C01CB1D4FEA00614FEA102099
:1006900042BF002010BC704700EBC350104400293B
:1006A000A4BF10BC7047401C490008BF20F00100E7
:1006B00010BC704710B5141E73F1000408DA401C1A
:1006C00041F1000192185B411A4301D120F0010071
:1006D00010BD2DE9F04D92469B4611B1B1FA81F261
:1006E00002E0B0FA80F220329046FFF77BFF04462A
:1006F0000F4640EA0A0041EA0B0153465A460843B6
:1007000013D0114653EA010019D0C8F140025046F7
:10071000FFF777FF05460E46504659464246FFF71B
:1007200061FF084305D0012004E020463946BDE8BA
:10073000F08D0020054346EAE0762C4337430A98C3
:100740006305E40AA0EB08000022FD0A44EA4754CE
:100750000A3002D500200146E9E701051019694178
:10076000DDE9084500196941BDE8F04DA2E7C1F394
:100770000A52C1F3130140F2FF3341F480119A424F
:1007800002DA00200146704740F233439A42A2F257
:10079000334202DC5242FFF734BFFFF723BF0000B1
:1007A00030B5041E71F1000404DB4FF000444042F8
:1007B00064EB0101141E73F1000405DB1C464FF0CD
:1007C0000043524263EB0403994208BF904230BD9C
:1007D000064C074D06E0E06840F0010394E807008E
:1007E00098471034AC42F6D3FFF7D2FCE42A010854
:1007F000042B0108464910B54A6822F440324A6089
:100800004A6843681A434A6001684A6822F4807261
:100810004A6001684A68036942EA03224A60016843
:100820004A6822F040724A6001684A6883681A4345
:100830004A6001688A6822F400628A6001688A68F6
:10084000C3681A438A60816A6FF07062D14201689E
:100850008A6822F070628A6001688A680CD0836AB4
:100860001A438A6001688A6822F040528A600168EF
:100870008A68C36A1A4301E022F040528A60016824
:100880008A6822F002028A6001688A68037E42EA6E
:1008900043028A6090F82010002901684A680FD04E
:1008A00042F400624A6001684A6822F460424A6089
:1008B00001684A68174C436A04EB43331A4301E06A
:1008C00022F400624A600168CA6A22F47002CA62B5
:1008D0000168CA6A838B104C04EB03531A43CA6243
:1008E00001688A6822F400728A6001688A6890F858
:1008F000303042EA43228A6001688A6822F48062CA
:100900008A6001688A68406942EA8020886010BD78
:100910000023014000E0FFFF0000F0FFFEE770470A
:100920007047000078B50024009490F83C20012A1C
:1009300019D0012280F83C200A6807230568092A9B
:1009400013D9EE680A3A02EB420293409E43EE60EE
:100950000B788A680A3B03EB43039A400368DD681F
:100960002A43DA6010E0022078BD2E6902EB4202D1
:1009700093409E432E610B788A6803EB43039A40B1
:1009800003681D692A431A614A681F23072A13D284
:1009900005686E6B521E02EB820293409E436E63AB
:1009A0000B790A885B1E92B203EB83039A400368BB
:1009B0005D6B2A435A6327E005680D2A12D22E6B1D
:1009C000D21F02EB820293409E432E630B790A886A
:1009D000DB1F92B203EB83039A4003681D6B2A432B
:1009E0001A6311E0EE6A0D3A02EB820293409E43D5
:1009F000EE620B790A880D3B92B203EB83039A40B7
:100A00000368DD6A2A43DA62164B0568144A9D4280
:100A100006D10D68122D03D1556845F48005556047
:100A200005689D4218D10B68102B01D0112B13D1F2
:100A3000536843F400035360096810290CD10A4934
:100A40000A4A0968B1FBF2F101EB8101490000E0BB
:100A5000491E00910029FBD180F83C40002078BD60
:100A600000230140002001402400002040420F00EC
:100A7000006C70470068C06C704770B504004FF0A0
:100A8000000503D0206C002610B107E0012070BDE6
:100A9000204600F01DF8666484F83C60206CC006B7
:100AA00010D4206C20F4885040F0020020642046CE
:100AB000FFF7A0FE6664206C20F0020040F0010009
:100AC000206400E0012584F83C60284670BD0000E9
:100AD00010B586B0044614216846FFF7ABFB1149F8
:100AE000206888421CD110480021026842F48072BC
:100AF0000260006800F4807005900B4814380268AA
:100B000042F001020260006800F001000590102030
:100B100000900320CDE901016946044800F0F4F893
:100B200006B010BD002001404438024000000240E1
:100B30002DE9F041044600680D4681684FF000073A
:100B400049050BD58068C00508D5206C40F0200011
:100B5000206484F83C700120BDE8F08100F0B2F917
:100B600006460FE0681C0DD025B100F0ABF9801BE4
:100B7000A84207D9206C40F00400206484F83C703F
:100B80000320E9E7206800688007EBD521686FF053
:100B900012000860206C40F40070206420688168B6
:100BA00011F0405F13D1217E89B9C16A11F4700F31
:100BB00002D0806840050AD4206C20F48070206444
:100BC000206CC00403D4206C40F00100206400209D
:100BD000C2E7000018B50021009190F83C20012ADE
:100BE00007D0012280F83C2002689368DB0702D01E
:100BF00011E0022018BD936843F0010393602A4A74
:100C00002A4B1268B2FBF3F202EB420200E0521EE2
:100C10000092002AFBD102689368DB0741D0036C85
:100C200040F20164A34343F48073036453685B059B
:100C300005D5036C23F4005343F480530364036C21
:100C4000DB0404D5436C23F00603436400E04164F5
:100C500080F83C1016496FF0220313604968006861
:100C6000CA06144906D088421BD1816811F0405F42
:100C700013D016E08842F8D00F4A904203D1D1F841
:100C80000423D206F1D00D4A90420AD1D1F80413C0
:100C900001F01F011029E8D303E0816841F0804191
:100CA0008160002018BD00002400002040420F0099
:100CB00000230140002001400021014000220140AA
:100CC00090F83510022903D080214165012070473A
:100CD000052180F835100068016821F001010160EC
:100CE0000020704770B5044600F0ECF80546601C23
:100CF00002D004480078044400F0E4F8401BA0420D
:100D0000FAD370BD180000202DE9F84FDFF87CB150
:100D100000224FF001084FF0030A4FF00F090BF1CA
:100D2000040E00BF0B6808FA02F42340A3426ED100
:100D30004D68022D01D0122D0ED1D50800EB850C87
:100D4000DCF820505607F70E09FA07F6B5430E698E
:100D5000BE402E43CCF82060066855000F790AFA91
:100D600005FC07F0030726EA0C06AF40374307608F
:100D70004E68012E05D0022E03D0112E01D0122E66
:100D80000ED18668CF6826EA0C06AF4037438760ED
:100D90004668A6430C79C4F300149440344344607D
:100DA000C6688C6826EA0C06AC403443C4604C68C4
:100DB000E40065D5364C256845F4804525602468F7
:100DC00022F0030504F480440094324C2E19D6F826
:100DD000084895072F0F09FA07F5AC432E4DA84296
:100DE00001D1002524E02D4DA84201D101251FE0AD
:100DF0002B4DA84201D102251AE02A4DA84201D16B
:100E0000032515E0284DA84202D1042510E037E063
:100E1000264DA84201D105250AE0254DA84201D161
:100E2000062505E0234DA84201D1072500E008254D
:100E3000BD402543C6F80858DBF800405D464E68C3
:100E40009C43F60300D51C432C60DEF80040754639
:100E50004E689C43B60300D51C432C600B4D0835EF
:100E60002C684E689C43F60200D51C432C60074D4D
:100E70000C352C684E689C43B60200D51C432C6090
:100E8000521C102AFFF44EAFBDE8F88F003C014021
:100E9000443802400030014000000240000402409B
:100EA00000080240000C0240001002400014024002
:100EB00000180240001C02400AB181617047090419
:100EC000FBE7000001488068704700001800002020
:100ED0000248816802781144816070471800002040
:100EE0000B4810B5016841F400710160016841F4DC
:100EF00080610160016841F480710160032000F0AD
:100F00006FF8002000F006F800F024F8002010BD73
:100F1000003C024070B50D4D04464FF47A712878BC
:100F2000B1FBF0F00A490968B1FBF0F000F0E2FA19
:100F300048B9102C07D200222146501E00F030F88C
:100F400000206C6070BD012070BD00001800002002
:100F5000240000200A4808B5016841F4804101607E
:100F6000006800F4804000900548001F016841F0CF
:100F700080510160006800F08050009008BD0000C2
:100F800044380240002809DB00F01F020121914093
:100F90004009800000F1E020C0F800117047000017
:100FA000F0B40E4B1B680C46C3F30223C3F10705D4
:100FB000042D00D90425191D072901D2002300E0C2
:100FC000DB1E012606FA05F1491E214099409E408C
:100FD000761E16403143F0BC01F00CB80CED00E079
:100FE000064900F0070208684FF6FF03184040EA80
:100FF0000220034A10430860704700000CED00E037
:101000000000FA052DE9F0470E46050065D0DFF82F
:101010001481D8F80000F7B200F00F00B04207D2F8
:1010200088F80070D8F8000000F00F00B04254D1EA
:1010300028683D4C810712D5400703D5206840F44D
:10104000E05020602878000703D5206840F4604015
:1010500020602068A96820F0F0000843206028780C
:10106000C0072DD0304968680839012812D00228FD
:1010700013D0032811D00968890700292DDA2168C7
:1010800021F0030101432160FFF71CFF814641F27B
:10109000883A0EE009688903EFE709688901ECE7FF
:1010A000FFF710FFA0EB0901514502D90320BDE86D
:1010B000F0872068696800F00C00B0EB810FEFD179
:1010C000D8F80010404601F00F01B14207D907706F
:1010D000006800F00F00B04201D00120E7E7287857
:1010E000400705D52068E96820F4E05008432060F7
:1010F0002878000706D52068296920F4604040EA76
:10110000C100206000F036F82168084AC1F30311DD
:10111000515CC840064908600020FFF7FBFE002034
:10112000C5E70000003C024008380240CC2A010814
:10113000240000200448054900680968044AC1F3F6
:101140008221515CC84070472400002008380240CA
:10115000DC2A01080448054900680968044AC1F30B
:101160004231515CC84070472400002008380240DA
:10117000DC2A0108154810B5006810F00C0214486C
:1011800013D01449042A0FD0082A0ED10F4C241F63
:101190002268236802F03F025B0207D52068C0F393
:1011A0008810A0FB010106E0084610BD2168C1F3CC
:1011B0008811A1FB00010023FFF704F82168C1F3A7
:1011C0000141491C4900B0FBF1F010BD0838024054
:1011D0000024F40040787D012DE9F84F050076D019
:1011E0002878DFF8F8B2BE4CC00749D0DBF8001011
:1011F0005846C1F38101012908D00068C0F381007D
:1012000002280AD1201D0068400206D5206880030C
:1012100036D568680028E2D032E06868B0F5803FD3
:1012200010D0B0F5A02F206810D020F480302060BE
:10123000206820F4802020606868A0B1FFF742FE9B
:1012400006460CE0206840F48030F4E740F480204B
:101250002060F7E7FFF736FE801B642873D820680C
:101260008003F7D50CE0FFF72DFE064605E000BF32
:10127000FFF728FE801B6428F0D820688003F7D48D
:101280002878DFF8608280074FF000093ED5DBF850
:101290000010584611F00C0F09D00068C0F381000F
:1012A00002280BD18D48001F0068400206D4206838
:1012B000800715D5E868012809D111E0E868B8B1C0
:1012C0000120C8F80000FFF7FDFD064605E002E139
:1012D000FFF7F8FD801B0228C0D820688007F7D5EB
:1012E0002068296920F0F80040EAC10020600DE084
:1012F000C8F80090FFF7E6FD064604E0FFF7E2FDC0
:10130000801B02281FD820688007F7D428780007A0
:1013100022D5724E744869696C3671B10121016041
:10132000FFF7D0FD074604E0FFF7CCFDC01B022805
:1013300009D830688007F7D50EE0C0F80090FFF7B5
:10134000C1FD074605E083E0FFF7BCFDC01B022896
:101350007ED830688007F7D42878400768D5DFF852
:101360007CA100270AF1380ADAF80000C0000BD48B
:10137000DAF8001041F08051CAF80010DAF80000E5
:10138000012700F080500090584E3068C00510D4FE
:10139000306840F480703060FFF794FD009005E005
:1013A000FFF790FD0099401A022851D83068C00517
:1013B000F6D54A4EA868683601280FD0052830684F
:1013C00010D020F001003060306820F00400306060
:1013D000A868B8B1FFF776FD00900FE0306840F0E4
:1013E0000100F4E740F004003060F7E7FFF76AFD22
:1013F0000099411A41F28830814264D830688007F0
:10140000F4D50EE0FFF75EFD009007E0FFF75AFD10
:101410000099411A41F28830814254D830688007DF
:10142000F4D42FB1DAF8001021F08051CAF800107E
:10143000A869C0B3DBF80010C1F3810102294AD0CA
:101440000228484607D0C8F86000FFF73BFD00E0DF
:1014500039E005463AE04746C8F86000FFF732FD3C
:10146000064604E0FFF72EFD801B02282BD82068DB
:101470008001F7D4D5E907010843A96A1C4A490845
:1014800002EB01416A6A41EA8211084395F82C1087
:1014900040EA01611148001F016001203866FFF732
:1014A00011FD054605E014E0FFF70CFD401B022886
:1014B00009D820688001F7D50BE000BFFFF702FDD7
:1014C000401B022802D90320BDE8F88F2068800164
:1014D000F4D40020F8E70120F6E7000008380240C5
:1014E0000038024000004742800E47420070004032
:1014F0000000FFFF10B5401EB0F1807F01D3012036
:1015000010BD4FF0E02460610F21601700F072FD04
:101510000020A06107202061002010BD704700005E
:1015200070B5026804461068D168536910F00F0F57
:1015300050D003F0010501F4907635435DD0C20729
:1015400005D0CA0503D5E26B42F00102E26342070F
:1015500005D5DA0703D0E26B42F00202E2638207AC
:1015600005D5DA0703D0E26B42F00402E26302071A
:1015700005D5DA0703D0E26B42F00802E263E26BC2
:10158000002A33D0800604D5880602D5204600F014
:101590000DFB20684069E16BC0F38010090700D49F
:1015A00028B3204600F0F4FA2068416949061AD5AC
:1015B000416921F040014161606BA0B11B490165A7
:1015C000606BFFF77DFB002810D0606B016DBDE8FC
:1015D00070400847830610D58B060ED52046BDE81F
:1015E000704000F0E3BA2046FFF798FF70BD204638
:1015F000FFF794FF0020E06370BD030606D50B06DD
:1016000004D52046BDE8704000F072BC4006F3D51A
:101610004806F1D5D168204621F04001D160202153
:1016200084F8391000F01CF970BD0000811B01081E
:1016300070B5040004D094F83900002510B106E01C
:10164000012070BD84F83850204600F023F8242093
:1016500084F839002068C16821F40051C160204637
:1016600000F0F0FA2068016921F4904101612068DE
:10167000416921F02A0141612068C16841F40051AB
:10168000C160E563202084F8390084F83A00002026
:1016900070BD0000F0B587B0044614216846FEF71F
:1016A000C9FD3A48384E25683849103802220123CE
:1016B0000324B5421FD10D6845F400250D6009686B
:1016C00001F400210591016841F004010160006806
:1016D000694600F004000590A0028DE81D00082076
:1016E00004902B48FFF710FB002211463420FFF72F
:1016F00057FC342022E0274F0726BD4222D1234940
:10170000091D0D6845F010050D60096801F0100114
:101710000591016841F0020101600068694600F02E
:1017200002000590C0208DE85D001B48FFF7ECFA31
:10173000002211462520FFF733FC2520FFF722FC6D
:1017400007B0F0BD154FBD42FAD10D6845F4003524
:101750000D60096801F400310591016841F008014C
:1017600001600068694600F00800059060208DE87F
:101770005D000B48FFF7C8FA002211462620FFF74C
:101780000FFC2620DAE70000004C00404038024001
:1017900000080240001001400004024000440040E4
:1017A000000C024070472DE9F843044690F83900D8
:1017B0001F4616460D46202850D1A5B19EB194F87B
:1017C000380001284AD0012084F838004FF0000882
:1017D000C4F83C80212084F83900FFF773FBA6840D
:1017E0008146E68426E00120BDE8F883E08C401EB7
:1017F000E084A0684B46B0F5805F4FF000024FF0E8
:1018000080012046009703D000F0A3FBE8B90DE06B
:1018100000F09FFBC8B928882168C0F30800486021
:10182000206908B16D1C05E0AD1C03E0216815F8C6
:10183000010B4860E08C0028D8D14B4600224021A3
:101840002046009700F085FB08B10320CCE720205C
:1018500084F8390084F838800020C5E70220C3E707
:101860007047FEE77FB50024144800940194029469
:1018700011490394C0E9001484600461047680F87F
:1018800020400F49C0E90A140125C561C46080F8F1
:1018900030404561FFF7F1F808B1FFF741F8042047
:1018A000CDE90005694602940448FFF73BF800289B
:1018B00001D0FFF735F87FBD002001402C0000204B
:1018C0000100000F2DE9F04F87B014216846FEF7A4
:1018D000B1FC3F480024016841F00101016001684A
:1018E00001F001010591016841F0100101600168FA
:1018F00001F010010591016841F0020101600168E9
:1019000001F002010591016841F0080101600168E0
:1019100001F008010591016841F0040101600068CF
:10192000DFF8B0A000F004004FF4784505900122E4
:1019300029465046FFF7C0FADFF89CB04FF4404606
:10194000012231465846FFF7B7FA4FF47C4701228F
:1019500039462248FFF7B0FA4FF400780122414699
:101960001F48FFF7A9FA4FF47C59012249461D4848
:10197000FFF7A2FA00950125CDE9015469465046CA
:101980000394FFF7C1F90096CDE901546946584622
:101990000394FFF7B9F90097CDE9015469460F4860
:1019A0000394FFF7B1F9CDF80080CDE90154694601
:1019B0000B480394FFF7A8F9CDF80090CDE9015446
:1019C000694608480394FFF79FF907B0BDE8F08F18
:1019D000303802400010024000040240000C024077
:1019E00000080240000002400C4810B50A4901609E
:1019F0004FF4E1314160002181600C22C160C0E9F7
:101A000004128161C161FFF713FE002803D0BDE815
:101A10001040FEF785BF10BD004C00407400002050
:101A20000C4810B50A4901604FF4E13141600021D2
:101A300081600C22C160C0E904128161C161FFF7BD
:101A4000F7FD002803D0BDE81040FEF769BF10BDC8
:101A500000100140B40000200C4810B50A49016094
:101A60004FF416414160002181600C22C160C0E941
:101A700004128161C161FFF7DBFD002803D0BDE8DE
:101A80001040FEF74DBF10BD00440040F4000020A0
:101A9000FEE7704770477047FFF71ABA30B593B04A
:101AA00030216846FEF7C6FB14210CA8FEF7C2FBE6
:101AB00018480025016841F080510160006800F07D
:101AC000805011901448016841F480410160006821
:101AD000022400F480401190012003901020049013
:101AE000009406940820CDE907504820CDE9090468
:101AF00003200B906846FFF76FFB0CA90F2081E8CD
:101B00003100E002CDE90F0502210CA8FFF77AFAB7
:101B100013B030BD403802400070004010480168EA
:101B200041F4700101600F48016841F0010101605A
:101B30000C4A00210832116002680B4B1A40026007
:101B4000031D0A4A1A60026822F4802202600548D6
:101B50000C30016002490648803908607047000077
:101B600088ED00E000380240FFFFF6FE1030002450
:101B7000000001080148FFF7D3BC000074000020FA
:101B800010B5806B0021C185C184FFF7C7FC10BD73
:101B90000168CA6822F49072CA6001684A6922F03A
:101BA00001024A61202180F83A10704710B590F880
:101BB0003A10222901D0022010BD8168B1F5805F62
:101BC00011D00169002901681FD0496801F07F0325
:101BD000816A4A1C82620B70C18D491E0904090C7E
:101BE000C18518D02BE00269816A002A0268526818
:101BF00005D0D2B20A80816A491C8162ECE7C2F347
:101C000008020A80816A891CF7E74A68816A4B1CCE
:101C100083620A70E0E70168CA6822F02002CA60A5
:101C20000168CA6822F48072CA6001684A6922F0B9
:101C300001024A61202180F83A10FFF7B3FD00202D
:101C400010BD00002DE9F041044600680169E2681A
:101C500021F44051114301612169A068E269084300
:101C60006169114322680843D16849F20C639943C2
:101C70000143D16020684169A26921F44071114398
:101C80004161E2696425B2F5004F9748974922689F
:101C90004FF032083FD08A4201D082427CD1FFF718
:101CA00059FA00EBC00101EB001061688900B0FB3C
:101CB000F1F6FFF74FFA00EBC00101EB001061688D
:101CC0008900B0FBF1F0B0FBF5F06FF0180148436C
:101CD00006EB800108EB0110B0FBF5F000F0F00618
:101CE000FFF738FA00EBC00101EB001061688900D2
:101CF000B0FBF1F0B0FBF5F006EB0016FFF72AFAA7
:101D000000EBC00101EB001061688900B0FBF1F746
:101D1000FFF720FAD2E08A4201D082423DD1FFF79C
:101D200019FA00EBC00101EB001061684900B0FB3B
:101D3000F1F0B0FBF5F00601FFF70CFA00EBC00183
:101D400001EB001061684900B0FBF1F7FFF702FA00
:101D500000EBC00101EB001061684900B0FBF1F03D
:101D6000B0FBF5F06FF01801484307EB800108EB7A
:101D7000C100B0FBF5F000F0F80006EB4006FFF7FD
:101D8000E9F900EBC00101EB001061684900B0FB0C
:101D9000F1F7FFF7DFF93CE055E0FFF7CBF900EB97
:101DA000C00101EB001061684900B0FBF1F0B0FB2D
:101DB000F5F00601FFF7BEF900EBC00101EB0010E2
:101DC00061684900B0FBF1F7FFF7B4F900EBC0011F
:101DD00001EB001061684900B0FBF1F0B0FBF5F0D9
:101DE0006FF01801484307EB800108EBC100B0FB1E
:101DF000F5F000F0F80006EB4006FFF79BF900EB6A
:101E0000C00101EB001061684900B0FBF1F7FFF77A
:101E100091F900EBC00101EB001061684900B0FBD3
:101E2000F1F0B0FBF5F06FF01801484307EB8001CB
:101E300008EBC100B0FBF5F000F00700216830446A
:101E40008860BDE8F081FFF775F900EBC00101EB98
:101E5000001061688900B0FBF1F6FFF76BF900EB49
:101E6000C00101EB001061688900B0FBF1F0B0FB2C
:101E7000F5F06FF01801484306EB800108EB011004
:101E8000B0FBF5F000F0F006FFF754F900EBC001ED
:101E900001EB001061688900B0FBF1F0B0FBF5F0D8
:101EA00006EB0016FFF746F900EBC00101EB00104E
:101EB00061688900B0FBF1F7FFF73CF900EBC00166
:101EC00001EB001061688900B0FBF1F0B0FBF5F0A8
:101ED0006FF01801484307EB800108EB0110B0FBDD
:101EE000F5F000F00F00A9E70014014000100140D8
:101EF00090F83910212901D0022070478168B1F58E
:101F0000805F016A0BD04A1C026202680978516046
:101F1000C18C491E0904090CC1840ED017E0098840
:101F20000268C1F30801516001690029016A02D009
:101F3000491C0162ECE7891CFBE70168CA6822F0D2
:101F40008002CA600068C16841F04001C1600020A1
:101F500070472DE9F041984617460E460446069D07
:101F60001DE0681C1BD02DB1FEF7ACFFA0EB0800F4
:101F7000A84214D92068C16821F4D071C1602068DA
:101F8000416921F001014161202084F8390084F881
:101F90003A00002084F838000320BDE8F081206872
:101FA000006836EA000004D00020B842D9D00020F2
:101FB000F3E70120F9E700000148FFF7B1BA00009C
:101FC000B40000200148FFF7ABBA0000F400002085
:101FD000FEE700000FB4054B10B503A9044A0298B0
:101FE00000F0EAF810BC5DF814FB0000C1280108FD
:101FF000280000200907090E002804DB00F1E0207A
:1020000080F80014704700F00F0000F1E02080F825
:10201000141D704702E008C8121F08C1002AFAD137
:1020200070477047002001E001C1121F002AFBD158
:10203000704700002DE9FF5F82B00021DDE9043028
:10204000020DDDF840B0034318D044F61050A2F260
:10205000FF3242431514119801281FD0A5EB0B0045
:10206000401C5FEA000A4FF000064E4FDFF838913F
:10207000B046504615D5CAF1000413E0119801246A
:102080004AA3012801D16FEA0B010298119AC0E915
:102090000031C0E9024206B0BDE8F09FCBF100007C
:1020A000DFE704460021404A491842EB0450CDE9DD
:1020B000001012E0E00707D032463B464046494652
:1020C000FEF76AF98046894632463B461046194675
:1020D000FEF762F906460F466410002CEAD1DDE9EE
:1020E0000401DDE90023BAF1000F06DAFEF754F926
:1020F00042464B46FEF750F905E0FEF7BFF942466F
:102100004B46FEF7BBF904460E460022284BFEF76D
:1021100047FB03D84FF0FF30014607E00022254B74
:1021200020463146FEF791F8FEF721FB102409E026
:10213000002C0ADB0A220023FEF744F8039B30320E
:102140001A55641E50EA0102F2D1641C039AC4F1CC
:1021500011031444119A012A03D0012208430DD11E
:102160000AE0084304D000204FF0110B119072E7F1
:10217000A3EB0B056D1E0DE05B4504DD4FF0000287
:1021800005F1010504E003DA4FF00002A5F10105B5
:10219000002AECD002981199C0E90231C0E900454B
:1021A00079E70000000014400000F03F300000001C
:1021B0000000F0430000E03F2DE9FF4F95B09A4644
:1021C000884606460025EEE1252877D100242746DB
:1021D000F94A0121039400E0044316F8013F203B33
:1021E00001FA03F01042F7D130782A2811D06FF0AD
:1021F0002F033078A0F13002092A16D8039A44F050
:10220000020402EB820203EB42021044761C0390AC
:10221000EFE758F8042B0392002A03DA504244F403
:102220000054039044F00204761C30782E2816D116
:1022300016F8010F44F004042A280DD06FF02F0285
:102240003078A0F13003092B09D807EB870302EBA4
:102250004303C718761CF3E758F8047B761C3078E4
:102260006C280FD006DC4C2817D068280DD06A28BF
:1022700014D104E0742810D07A280FD10DE044F472
:1022800000140AE044F4801401E044F4401472782D
:10229000824202D104F58014761C761C30786628C0
:1022A0000BD013DC582877D009DC002875D04528DE
:1022B000F6D04628F4D047281AD193E118E06328D5
:1022C00035D0642879D0652812D18BE1702873D07D
:1022D00008DC6728F1D069286FD06E280DD06F28F0
:1022E00006D1ACE073282CD0752874D0782853D050
:1022F0005246179990476D1C54E1C4F302500228CE
:1023000009D003280DD0D8F8001004280DD00D6096
:1023100008F1040846E1D8F80010EA17C1E90052B4
:10232000F6E7D8F800100D80F2E70D70F0E718F826
:10233000041B8DF8001000208DF80100EB460120F1
:1023400003E058F804BB4FF0FF3061074FF0000185
:1023500002D40DE009F101018946B9420FDA814545
:10236000F8DB1BF809100029F4D108E009F101019C
:1023700089468142FADB1BF809100029F6D103983F
:102380005346A0EB090721463846179A00F080FA19
:10239000284400EB090507E044E008E10DE01BF8E4
:1023A000010B524617999047B9F10109F7D25346EC
:1023B00021463846179AF2E039E00A21C4F3025266
:1023C0004FF0000B0091022A06D058F8040BC117F9
:1023D000032A09D00AE023E008F1070020F00702F1
:1023E000F2E80201904605E000B2C117042A01D1CB
:1023F00040B2C117002906DA0A460021404261EBCB
:1024000002012D2202E0220504D52B228DF80420A2
:10241000012203E0E20701D02022F7E7914657E0CE
:102420000A2100E010214FF0000B00910BE0102179
:102430004FF0000B44F004040827009103E008204B
:102440004FF0000B0090C4F30252022A05D058F856
:10245000040B0021032A08D008E008F1070020F04F
:102460000702F2E80201904603E080B2042A00D19C
:10247000C0B24FF0000922072AD53278702A07D05F
:10248000DDF800C08CF0100C5CEA0B0C05D00EE0FF
:1024900040228DF80420012208E050EA010306D012
:1024A00030238DF804308DF8052002229146009BE0
:1024B00083F0080353EA0B030AD150EA010201D169
:1024C000620705D530228DF804204FF001097F1EE8
:1024D0003278582A04D039A20C920CAA02920BE04E
:1024E0003BA2F9E75B46009AFDF76CFE0C9B9B5CF8
:1024F000029A521E0292137050EA0102F2D102981F
:1025000004A9081A00F1200B600702D524F48034D6
:1025100000E001275F4502DDA7EB0B0000E0002093
:1025200000EB0B01009003984944401A0390E0032C
:1025300006D453462146179A039800F0A9F905449A
:10254000002706E001A85246C05D179990476D1C10
:102550007F1C4F45F6DBE0030CD553462146179A06
:10256000039800F095F9054404E03020524617998D
:1025700090476D1C0099481E00900029F5DC08E08A
:102580000298029952460078491C02911799904787
:102590006D1CBBF10001ABF1010BF1DC5BE100F064
:1025A00065F90544761C307800287FF40DAE19B02B
:1025B0002846BDE8F08F0000092801003031323391
:1025C000343536373839616263646566000000006F
:1025D0003031323334353637383941424344454659
:1025E00000000000600700D4062708F1070020F073
:1025F0000700F0E80223804603F0004C5FEA0C007D
:1026000001D097A009E0200501D596A005E0E007DC
:1026100001D095A001E0AFF24C001390307823F088
:10262000004365280CD006DC452809D046281DD07B
:1026300047287FD13BE0662818D067287AD136E05A
:102640000021112F01DB112000E0781CCDE90001F1
:1026500004A90CA8FFF7EEFCDDE90D010C9A4FF080
:10266000000B07F10109109200914EE04FF000407D
:102670000097CDE9011004A90CA8FFF7DBFCDDE908
:102680000D020C9B0F994FF0000B91461093009296
:1026900011B9791C00EB0109B7EB090003D4C0F1B3
:1026A000FF3B07F10109A9EB0700019042E0012F70
:1026B00000DA01270021112F01DD112000E038464A
:1026C000CDE9000104A90CA8FFF7B4FCDDE90D0178
:1026D0000C9A00914FF0000BB946109221070FD4CD
:1026E000009A4A4503DA914601E0A9F10109B9F1DE
:1026F000010F05DD109AA9F10101515C3029F4D0D8
:10270000B84202DA10F1040F03DA0121CDE9011019
:1027100010E0002803DC8344A9EB000102E0411C27
:10272000494500DD8946A0EB0B00401C01904FF0AD
:1027300000400290200705D40198484502DB4FF085
:10274000FF30019000208DF84B0002980DF14B07EF
:10275000B0F1004F25D002200C902B200D90029854
:1027600000280CDA404202902D200D9007E00A214B
:102770000298FDF721FF3031029007F8011D0C99F6
:10278000481E0C900029F2DC02980028EFD1791E37
:102790000D980870307800F0200040F0450007F8F0
:1027A000020D11A8C01BC01D02901398007800B143
:1027B000012000EB0901019801EBE071029801444E
:1027C0000398401A401E0390E00306D45346214666
:1027D000179A039800F05CF805441398007818B134
:1027E0005246179990476D1CE00323D55346214666
:1027F000179A039800F04CF805441BE0BBF1000F5A
:1028000007DB0098584504DD1098179910F80B0065
:1028100001E0179930205246904701980BF1010BC7
:10282000401E05F10105019004D12E205246179952
:1028300090476D1CB9F10001A9F10109DEDC05E04A
:1028400017F8010B5246179990476D1C0299481EC4
:1028500002900029F4DC53462146179A03989EE61D
:102860002D0000002B000000200000002DE9F041A9
:10287000044600251E461746880404D405E0394660
:102880002020B0476D1C641EF9D52846BDE8F081B4
:102890002DE9F041044600251E469046C80301D5A7
:1028A000302700E02027880404D505E0414638465B
:1028B000B0476D1C641EF9D52846BDE8F0810000C4
:1028C00001B54FF6FF73012269460248FEF76BFF20
:1028D000009808BD740000202DED088BFEF700FB6A
:1028E000FFF7DCF8FEF7EEFFFFF7B6F8FFF77CF82E
:1028F000FFF796F8FEF7B6FF9FED55AB9FED56BB81
:10290000574CDFF8608142F210795748FEF762F9C0
:1029100032215548FEF70CF95348FEF7A9F8800517
:1029200062D55148FEF7A6F880B200EE100A20806A
:10293000B8EE400A9FED4D8A20EE080ADFED4C8A82
:1029400020EE280A10EE100AFDF707FE41EC100BEE
:1029500048A053EC102BFFF73DFB208800EE100A37
:10296000B8EE400A20EE080A20EE280A84ED010A9B
:1029700094ED028AB4EEC80AF1EE10FA30EE480A7D
:1029800010EE100A08DDFDF7E8FD94ED030A41ECB6
:10299000190B30EE480A07E0FDF7DFFD94ED040A5D
:1029A00041EC190B38EE400A10EE100AFDF7D5FD88
:1029B00041EC100B51EC1A0B53EC102BFDF75EFDA4
:1029C00053EC192BFDF7E8FC53EC1B2BFDF7E1FC56
:1029D000FDF7D6FD6061FDF7C0FD41EC100B2AA0AC
:1029E00053EC102BFFF7F6FA4846FEF77BF96069C7
:1029F00040458ADC284E4FF40055002229463046D7
:102A0000FEF75AFA25A0FFF7E5FA6F1000223946C3
:102A10003046FEF751FA24A0FFF7DCFA4FF4FA70C3
:102A2000FEF760F9012239463046FEF745FA21A04B
:102A3000FFF7D0FA4FF47A70FEF754F901222946D5
:102A40003046FEF739FA1EA0FFF7C4FA5DE7000032
:102A500000000000000008400000000000001C40D2
:102A6000000000200000C8412C00002033335340F8
:102A700000008039766F6C74616765203A202531DB
:102A80002E3366560A0000004D345F50483A202528
:102A9000312E31660A0000000000024072656C6150
:102AA00079313A310A00000072656C6179323A314D
:102AB0000A00000072656C6179323A300A00000049
:102AC00072656C6179313A300A0000000000000044
:102AD00000000000010203040607080900000000CE
:102AE00001020304042B0108000000202C00000058
:102AF00014200108302B01082C0000200C4100009C
:102B00002420010800000000000000000000C03F79
:102B100085EB01409A99793F000000000100000018
:102B200010000000000000000024F400000000007D
:040000050801018964
:00000001FF
